:100000000C94340018950000189500001895000015
:10001000189500001895000018950000189500002C
:10002000189500001895000018950000189500001C
:10003000189500001895000018950000189500000C
:1000400018950000189500000C94B70E1895000044
:1000500018950000189500001895000018950000EC
:1000600018950000189500008FEF8DBFC0E8E8E9F3
:100070004E2E88E08EBFD8E0F7E05F2EA89584B7BB
:10008000082E877F84BF88E1992780936000909332
:100090006000EEEFF7E0A0E0B1E088278D933197A4
:1000A000E9F787E68093C40080E08093C50088E18B
:1000B0008093C1006624299A5E9A289A5F9A5C9A76
:1000C0005A9A439A559A539A2A9A229A419A399A55
:1000D0002D9A259A0E94500C389A399A3A9A239A66
:1000E000259A0E94760C0E94A10C70E07093B900D2
:1000F0007CE07093B8000E94710D87E880937A00CD
:1001000080E480937C0070917A00706870937A002C
:1001100087E68093C40080E08093C5007091C000A2
:100120007D7F7093C00088E18093C10086E080935A
:10013000C2007091C10070687093C100789480E033
:10014000809380008DE08093810088E09DE3909310
:10015000890080938800E8EBF2E1A0E0B1E0ED9344
:10016000FC930E94DB0BE8ECFEE10E94D40B0E94A2
:10017000DB0B539AE5E3F5E082E390E001975B9AAD
:100180000E945A0C5B980E945A0C482F492BB1F7D9
:100190005D9A80ED809360012CEE81E091E0A0E615
:1001A000B1E00E94D00D00916001003611F40C9472
:1001B000090182E08093020187E080930301882790
:1001C00080930401EEEFFEE10E94ED0B84E080934A
:1001D00002018DE08093030181E080930401E8E057
:1001E000FFE10E94ED0BE4E1FFE10E94D40B0E94CD
:1001F000DB0B539AEAE0FAE184E690E001975B9A20
:100200000E945A0C5B980E945A0C482F492BB1F758
:10021000FFCF0E943F02E4E1F5E1A0E0B1E0ED9301
:10022000FC9381E08093020181E08093030183E0ED
:1002300080930401EAE2FFE10E94ED0B81E08093EC
:10024000020189E48093030183E0809304018FE33A
:100250000E94F40B83E08093020181E0809303010C
:1002600083E080930401EAE2FFE10E94ED0B83E06A
:100270008093020189E48093030183E08093040169
:10028000E4E3FFE10E94ED0BE8EBF2E1A0E0B1E076
:10029000ED93FC9385E08093020189E48093030150
:1002A000882780930401E6E3FFE10E94ED0B86E0DE
:1002B0008093020189E480930301882780930401DD
:1002C000E8E3FFE10E94ED0BB19B0C942102B19A8F
:1002D0000E944003E4E1F5E1A0E0B1E0ED93FC937E
:1002E000E8E5F1E0AEE7B1E00E940B0FA8E5B1E070
:1002F0000D911C91003050E015070CF402C00C94D5
:10030000980181E0809302018BE08093030183E0F8
:1003100080930401EEE7F1E0A0E8B7E014E02227C3
:1003200003E032E00E94790E0E94E50B0C94AD01CF
:1003300081E0809302018BE08093030183E080934E
:100340000401EEE7F1E0A0E8B7E015E0222703E0C2
:1003500032E00E94790E0E94E50BECE3FFE10E947F
:10036000D40BEEE7F1E0A0E8B7E014E0222703E0C9
:1003700032E00E94790E0E94CC0BECE4FFE10E9477
:10038000D40BEAE5F1E0AEE7B1E00E940B0F83E0A9
:10039000809302018BE08093030183E0809304014A
:1003A000EEE7F1E0A0E8B7E015E0222703E032E055
:1003B0000E94790E0E94E50BE2E5FFE10E94D40B5A
:1003C000EEE7F1E0A0E8B7E015E0222703E032E035
:1003D0000E94790E0E94CC0BEEE5FFE10E94D40B47
:1003E000ECE5F1E0AEE7B1E00E94080F85E0809314
:1003F000020181E080930301882780930401EEE7E6
:10040000F1E0A0E8B7E016E0222703E032E00E9426
:10041000790E0E94E50BE4E6FFE10E94D40BEEE7C3
:10042000F1E0A0E8B7E016E0222703E032E00E9406
:10043000790E0E94CC0BE0E7FFE10E94D40B0E94F2
:10044000DB0B3B98A3E9B1E09C9197FF04C0339B81
:1004500010C09F779C9333990CC089E19F9390E0E3
:100460000E94670C9F91339904C090689C930C94F0
:100470003B020C94640180E289B90C94640182EF20
:100480008093600185E08093610184EF8093620135
:1004900087EB8093630185EF8093640180EB809309
:1004A000650186E08A931CEEA0E6B1E00E94C50DCE
:1004B00088E8809360012CEE81E09AE1A0E6B1E04B
:1004C0000E94D00D9091610180916001A4E9B1E09A
:1004D0008D939C939091630180916201A6E9B1E0B4
:1004E0008D939C939091650180916401A8E9B1E09E
:1004F0008D939C939091670180916601AAE9B1E088
:100500008D939C939091690180916801ACE9B1E071
:100510008D939C9390916B0180916A01AEE9B1E05B
:100520008D939C9390916D0180916C01A0EAB1E054
:100530008D939C9390916F0180916E01A2EAB1E03E
:100540008D939C939091710180917001A4EAB1E028
:100550008D939C939091730180917201A6EAB1E012
:100560008D939C939091750180917401A8EAB1E0FC
:100570008D939C939091770180917601AAEAB1E0E6
:100580008D939C93A9E7B1E08C91ACEAB1E08D9397
:1005900088278C9381EE809360012CEE81E097E0B8
:1005A000A0E6B1E00E94D00D9091610180916001C0
:1005B000AEEAB1E08D939C93A2E6B1E08C91A0EB02
:1005C000B1E08D9388278C93A3E6B1E08C91A2EBE8
:1005D000B1E08D9388278C9394E0A2EBB1E00E9468
:1005E0002A0EA4E6B1E00D9111274FE050E004235C
:1005F0001523A4EBB1E00D931C93A2EBB1E00D9198
:100600001C91A4EBB1E04D915C91040F151FA2EB7E
:10061000B1E00D931C93A4E6B1E00D91112740EFDA
:1006200050E004231523A4EBB1E00D931C9394E058
:10063000A4EBB1E00E944A0EA5E6B1E08C91A6EBD6
:10064000B1E08D9388278C9394E0A6EBB1E00E94F3
:100650002A0EA4EBB1E00D911C91A6EBB1E04D91F7
:100660005C91040F151FA4EBB1E00D931C93A6E65B
:10067000B1E08C91A6EBB1E08D9388278C9308951F
:1006800087EF809360012CEE81E098E0A0E6B1E076
:100690000E94D00D9091600180916101A0EDB1E0C8
:1006A0008D939C93A0EDB1E08D919C91ACEBB1E06A
:1006B0008D939D9388278D938C9394E0ACEBB1E060
:1006C0000E94350E94E0A2E6B1E00E94420EACEB2F
:1006D000B1E00D911D912D913C91A2E6B1E04C91BC
:1006E0005527662777270E94E50EACEBB1E00D9306
:1006F0001D932D933D939091630180916401A0ED32
:10070000B1E08D939C93A0EDB1E08D919C91A8EB0D
:10071000B1E08D939D9388278D938C9394E0A8EB03
:10072000B1E00E94350E94E0A5E6B1E00E94420ED1
:10073000A8EBB1E00D911D912D913C91A5E6B1E0A2
:100740004C915527662777270E94E50EA8EBB1E06C
:100750000D931D932D933D939091660180916701B8
:10076000A0EDB1E08D939C93A0EDB1E08D919C91B3
:10077000A0ECB1E08D939D9388278D938C9393E0AB
:10078000A8EBB1E00E94550EA8EBB1E00D911D91D0
:100790002D913C91A4E9B1E04D915C9166277727BA
:1007A0000E94EA0EA4ECB1E00D931D932D933D93AE
:1007B000A4ECB1E00D911D912D913C91A4E9B1E023
:1007C0004D915C91662777270E94EA0EA4ECB1E078
:1007D0000D931D932D933D93A4ECB1E00D911D91CC
:1007E0002D913C91A6E9B1E04D915D9157FB1EF42E
:1007F0006FEF7FEF02C0662777270E94070EA4ECF9
:10080000B1E00D931D932D933D939BE0A4ECB1E0DB
:100810000E94620E91E0A8EBB1E00E94550EA8EB99
:10082000B1E00D911D912D913C91A4E9B1E04D9164
:100830005C91662777270E94EA0EA8ECB1E00D9341
:100840001D932D933D93A8ECB1E00D911D912D9139
:100850003C91A8ECB1E04D915D916D917C910E942D
:10086000070EA8ECB1E00D931D932D933D939CE0F2
:10087000A8ECB1E00E94620EA8ECB1E00D911D91D0
:100880002D913C91A8E9B1E04D915D9157FB1EF48B
:100890006FEF7FEF02C0662777270E94070EA8EC54
:1008A000B1E00D931D932D933D939EE0A8ECB1E034
:1008B0000E94620EA4ECB1E00D911D912D913C912E
:1008C000A8ECB1E04D915D916D917C910E94E50E97
:1008D000A2EDB1E00D931D932D933D93A2EDB1E0F8
:1008E0000D911D912D913C9145E050E060E070E04C
:1008F0000E94070EA8ECB1E00D931D932D933D933C
:10090000A8ECB1E00D911D912D913C9140E850E093
:1009100060E070E00E94E50EA8ECB1E00D931D933D
:100920002D933D9398E0A8ECB1E00E94620EA8ECF4
:10093000B1E08D919C91A8E5B1E08D939C93A2EDDF
:10094000B1E00D911D912D913C91A4ECB1E00D937E
:100950001D932D933C9391E0A4ECB1E00E94620EB4
:10096000A4ECB1E00D911D912D913C9140E05AEF26
:1009700060E070E00E94EA0EA4ECB1E00D931D93DC
:100980002D933D93A4ECB1E00D911D912D913C91DF
:10099000A8ECB1E00D931D932D933C9392E0A8EC4D
:1009A000B1E00E94620EA8ECB1E00D911D912D9175
:1009B0003C91A8ECB1E04D915D916D917C910E94CC
:1009C000070EA8ECB1E00D931D932D933D939BE092
:1009D000A8ECB1E00E94620EA8ECB1E00D911D916F
:1009E0002D913C91A4EAB1E04D915D9157FB1EF42D
:1009F0006FEF7FEF02C0662777270E94070EA8ECF3
:100A0000B1E00D931D932D933D93A4ECB1E00D91B6
:100A10001D912D913C91A2EAB1E04D915D9157FB62
:100A20001EF46FEF7FEF02C0662777270E94070E44
:100A3000ACECB1E00D931D932D933D9391E0ACECA4
:100A4000B1E00E94350EA8ECB1E00D911D912D9101
:100A50003C91ACECB1E04D915D916D917C910E9427
:100A6000E50EA8ECB1E00D931D932D933D93A0EA04
:100A7000B1E08D919C91ACECB1E08D939C930E9480
:100A8000EF0D90E1ACECB1E00E94350E92E0A8ECE5
:100A9000B1E00E94620EA8ECB1E00D911D912D9184
:100AA0003C91ACECB1E04D915D916D917C910E94D7
:100AB000E50EA8ECB1E00D931D932D933D93ACE9A9
:100AC000B1E00D911D9117FB1EF42FEF3FEF02C017
:100AD00022273327A4ECB1E04D915D916D917C917B
:100AE0000E94070EACECB1E00D931D932D933D9346
:100AF00091E0ACECB1E00E94620E92E0A4ECB1E0B7
:100B00000E94620EA4ECB1E00D911D912D913C91DB
:100B1000A4ECB1E04D915D916D917C910E94070E26
:100B2000A4ECB1E00D931D932D933D939DE0A4ECB7
:100B3000B1E00E94550EAEE9B1E00D911D9117FB99
:100B40001EF42FEF3FEF02C022273327A4ECB1E0C1
:100B50004D915D916D917C910E94070EA4ECB1E0E6
:100B60000D931D932D933D9393E0A4ECB1E00E946F
:100B7000620EA4ECB1E00D911D912D913C91ACEC75
:100B8000B1E04D915D916D917C910E94E50EA4ECD8
:100B9000B1E00D931D932D933D9392E1A4ECB1E050
:100BA0000E94620E00E010E820E030E0A4ECB1E02A
:100BB0004D915D916D917C910E94E50EA4ECB1E0A8
:100BC0000D931D932D933D93A4ECB1E00D911D91D8
:100BD0002D913C91AAE9B1E04D915C916627772770
:100BE0000E94070EA4ECB1E00D931D932D933D934D
:100BF0009FE0A4ECB1E00E94620E40E050E060E0B3
:100C000070E0A4ECB1E00D911D912D913C910E94FA
:100C1000EF0E11F00C94180600E010E020E030E038
:100C2000ACE5B1E00D931D932D933C930C946607B6
:100C300000E010E020E130E0ACEBB1E04D915D91DF
:100C40006D917C910E94EA0EACE5B1E00D931D938D
:100C50002D933D939CE0A8ECB1E00E94620EACE5C0
:100C6000B1E00D911D912D913C91A8ECB1E04D9119
:100C70005D916D917C910E94EA0EACE5B1E00D931F
:100C80001D932D933D93ACE5B1E00D911D912D91F8
:100C90003C9145E35CE060E070E00E94070EACE54B
:100CA000B1E00D931D932D933D9340E050E060E043
:100CB00070E8ACE5B1E00D911D912D913C910417C8
:100CC00015072607370710F00C94810691E0ACE574
:100CD000B1E00E94350EACE5B1E00D911D912D9172
:100CE0003C91A4ECB1E04D915D916D917C910E949D
:100CF000000CACE5B1E04D935D936D937D930C9446
:100D0000A906ACE5B1E00D911D912D913C91A4ECAB
:100D1000B1E04D915D916D917C910E94000CACE52C
:100D2000B1E04D935D936D937D93ACE5B1E00D9192
:100D30001D912D913C91ACE5B1E04D915D916D918E
:100D40007C910E94E50EACE5B1E00D931D932D93CF
:100D50003D93ACE5B1E00D911D912D913C91A4EC3A
:100D6000B1E00D931D932D933C9393E0A4ECB1E07F
:100D70000E94550EA4ECB1E00D911D912D913C9176
:100D8000A4ECB1E04D915D916D917C910E94070EB4
:100D9000A4ECB1E00D931D932D933D939DE0A4EC45
:100DA000B1E00E94550EAAEAB1E00D911D9117FB2A
:100DB0001EF42FEF3FEF02C022273327A4ECB1E04F
:100DC0004D915D916D917C910E94070EA4ECB1E074
:100DD0000D931D932D933D939CE0A4ECB1E00E94F4
:100DE000620EACE5B1E00D911D912D913C91A8EC06
:100DF000B1E00D931D932D933C9392E0A8ECB1E0EC
:100E00000E94550EA8ECB1E00D911D912D913C91E1
:100E1000A8EAB1E04D915D9157FB1EF46FEF7FEFB3
:100E200002C0662777270E94070EA8ECB1E00D9359
:100E30001D932D933D939DE0A8ECB1E00E94620EBE
:100E4000A4ECB1E00D911D912D913C91A8ECB1E085
:100E50004D915D916D917C910E94E50EA4ECB1E005
:100E60000D931D932D933D93A4ECB1E00D911D9135
:100E70002D913C91A6EAB1E04D915D9157FB1EF496
:100E80006FEF7FEF02C0662777270E94E50EA4EC84
:100E9000B1E00D931D932D933D9394E0A4ECB1E04C
:100EA0000E94620EACE5B1E00D911D912D913C9137
:100EB000A4ECB1E04D915D916D917C910E94E50EA5
:100EC000ACE5B1E00D931D932D933D93A2EDB1E000
:100ED0000D911D912D913C9140E05CE261E070E04C
:100EE0000E94EA0EA4ECB1E00D931D932D933D9367
:100EF000A0ECB1E00D911D912D913C91A8ECB1E0D9
:100F00000D931D932D933C939EE0A8ECB1E00E94BD
:100F1000350EA2EBB1E08D919C91ACECB1E08D93DC
:100F20009C930E94EF0D94E1ACECB1E00E94350E71
:100F3000A8ECB1E00D911D912D913C91ACECB1E08C
:100F40004D915D916D917C910E94EA0EA8ECB1E00B
:100F50000D931D932D933D93A4EBB1E00D911D9145
:100F600017FB1EF42FEF3FEF02C022273327A4EC1C
:100F7000B1E04D915D916D917C910E94070EACECBA
:100F8000B1E00D931D932D933D93A8ECB1E00D912D
:100F90001D912D913C91ACECB1E04D915D916D9125
:100FA0007C910E94EA0EA8ECB1E00D931D932D9365
:100FB0003D93A8ECB1E00D911D912D913C9140E045
:100FC00050E460E070E00E94E50EA8ECB1E00D9303
:100FD0001D932D933D939FE0A8ECB1E00E94620E1B
:100FE000A4ECB1E00D911D912D913C91A6EBB1E0E7
:100FF0004D915D9157FB1EF46FEF7FEF02C06627A6
:1010000077270E94070EACECB1E00D931D932D9352
:101010003D939AE0ACECB1E00E94620EA4ECB1E02A
:101020000D911D912D913C91A0EBB1E04D915C9102
:10103000662777270E94070EA2EDB1E00D931D935E
:101040002D933D939BE0A2EDB1E00E94620EA2EDD4
:10105000B1E00D911D912D913C9140E050E860E090
:1010600070E00E94E50EA2EDB1E00D931D932D936B
:101070003D93ACECB1E00D911D912D913C91A2ED11
:10108000B1E04D915D916D917C910E94070EACECA9
:10109000B1E00D931D932D933D939AE0ACECB1E03C
:1010A0000E94620EACECB1E00D911D912D913C912E
:1010B00040E050E060E270E00E94E50EACECB1E090
:1010C0000D931D932D933D93ACECB1E00D911D91CB
:1010D0002D913C91AEEAB1E04D915D9157FB1EF42C
:1010E0006FEF7FEF02C0662777270E94070EACECF8
:1010F000B1E00D931D932D933D93ACECB1E00D91B8
:101100001D912D913C9140E050E260E070E00E9422
:10111000E50EACECB1E00D931D932D933D939EE055
:10112000ACECB1E00E94620EA8ECB1E00D911D9113
:101130002D913C91ACECB1E04D915D916D917C9124
:101140000E94070EA4ECB1E00D931D932D933D93E7
:10115000A4ECB1E00D911D912D913C91ACECB1E06E
:101160000D931D932D933C939FE0ACECB1E00E9456
:10117000620EACECB1E00D911D912D913C91ACEC67
:10118000B1E04D915D916D917C910E94070EACECA8
:10119000B1E00D931D932D933D9397E0ACECB1E03E
:1011A0000E94620EACECB1E00D911D912D913C912D
:1011B000ACEAB1E04D915C91662777270E94070E5B
:1011C000ACECB1E00D931D932D933D9394E0ACEC0A
:1011D000B1E00E94620EA4ECB1E00D911D912D9141
:1011E0003C91ACECB1E04D915D916D917C910E9490
:1011F000EA0EA4ECB1E00D931D932D933D9340E0D6
:1012000050E060E070E0A4ECB1E00D911D912D91F3
:101210003C910E94EF0E0CF402C00C94190900E0FE
:1012200010E020E030E0A4ECB1E00D931D932D938D
:101230003C9340E050E060E079E1A4ECB1E00D9136
:101240001D912D913C910E94EF0E1CF011F00C9419
:101250002B090C94350900E010E020E039E1A4EC02
:10126000B1E00D931D932D933C939CE0A4ECB1E071
:101270000E94620EA4ECB1E00D911D912D913C9164
:1012800044E650E060E070E00E94070EA4ECB1E09C
:101290000D931D932D933D939AE0A4ECB1E00E9431
:1012A000620EA4ECB1E08D919C91AAE5B1E08D9322
:1012B0009C930895F894FFCF0106060000000000FB
:1012C00000000000005F000000000700070000149D
:1012D0007F147F1400242A7F2A12002313086462DB
:1012E00000364955225000000503000000001C2272
:1012F0004100000041221C000014083E08140008B0
:10130000083E0808000050300000000808080808DF
:10131000000060600000002010080402003E5149F7
:10132000453E0000427F400000625149494600228C
:1013300041494936001814127F10002745454539A8
:10134000003C4A494930000171090503003649490A
:10135000493600064949291E0000363600000000C3
:10136000563600000008142241000014141414140E
:101370000000412214080002015109060032497997
:10138000413E007E1111117E007F49494936003EE1
:1013900041414122007F4141221C007F494949418E
:1013A000007F09090901003E4149497A007F080888
:1013B000087F0000417F410000304040403F007FF7
:1013C00008142241007F40404040007F020C027F11
:1013D000007F0408107F003E4141413E007F090923
:1013E0000906003E4151215E007F09192946002669
:1013F000494949320001017F0101003F4040403F1F
:10140000000F3040300F001F601C601F0063140885
:101410001463000708700807006151494543000044
:101420007F4141000015167C1615000041417F00E8
:10143000000402010204004040404040000001025C
:101440000400002054545478007F48484830003845
:101450004444442800304848487F003854545418C5
:101460000000087E0901000C5252523E007F080421
:1014700004780000007D0000002040403D00007F17
:10148000102844000000007F4000007C04780478AD
:10149000007C08040478003844444438007C141468
:1014A000140800081414147C007C08040408004884
:1014B000545454200000043E4420003C4040207C12
:1014C000000C3040300C003C4038403C00442810B8
:1014D0002844000C5050301C004464544C4400001C
:1014E0000836410000000077000000004136080087
:1014F000000201020100007F7F7F7F7F10181C180F
:101500001000040C1C0C040000081C3E0000003EEF
:101510001C080000020A1400000000000000000087
:1015200000000000000000000000000000000000BB
:10153000FEFE000000000000000033330000000049
:1015400000001E1E00001E1E000000000000000023
:10155000000000000030F0FC3C30F0FC3C00003C9F
:101560003F0F0C3C3F0F0C000078FCCCFEFECCCCB7
:10157000880000040C0C3F3F0C0F07000030484867
:10158000B0C0E0703000000C0E07030D12120C000A
:1015900000009CFEE6BE1C000000001F3F31313BF6
:1015A0001F3F33000000004C7E3C000000000000A4
:1015B00000000000000000000000F0F80C0602002F
:1015C00000000000070F183020000000000000029B
:1015D000060CF8F000000000002030180F07000093
:1015E00000303040F8F840303000000606010F0FA0
:1015F0000106060000808080F0F0808080000001FD
:1016000001010F0F010101000000000000000000B7
:101610000000000000004C7E1C0000000080808064
:101620008080808080000001010101010101010032
:1016300000000000000000000000000000183C3C1A
:10164000180000000000000000C0F03C0C0000008A
:10165000303C0F030000000000F8FC0E06060EFCF4
:10166000F800000F1F383030381F0F000000181C22
:10167000FEFE00000000000030303F3F3030000030
:1016800000181C0E0686CEFC780000383C3E37332E
:101690003130300000181C0EC6C6EEFC3800000CBD
:1016A0001C383030391F0F0000C0E070381CFEFEBF
:1016B00000000007070606063F3F0600007E7E6624
:1016C0006666E6C68600000C1C383030381F0F00F6
:1016D00000E0F8DCCEC6C6860000000F1F393030AF
:1016E000391F0F00000606060686E67E1E00000073
:1016F00000383E07010000000038FCEEC6C6EEFCD4
:101700003800000F1F393030391F0F000078FCCE31
:101710008686CEFCF8000000003131391D0F030031
:10172000000000183C3C180000000000000C1E1EC9
:101730000C00000000000000183C18000000000031
:1017400000004C3E1C0000000080C0E070381C0C03
:101750000000000103070E1C38300000003030305C
:101760003030303030000006060606060606060059
:1017700000000C1C3870E0C08000000030381C0EE7
:10178000070301000C1212CCE0703070E0C00000C2
:10179000000F1F3830381C0CA0E8B7E08D9188236B
:1017A00011F00CD0FBCF08950E94750E802D11F022
:1017B00005D0FACF08958DE001D08AE00090C000F6
:1017C00005FEFCCF8093C6000895A0E8B7E08D9198
:1017D000882311F009D0FBCF08950E94750E802D4B
:1017E00011F002D0FACF08950C94AF0C00FC05D094
:1017F000089530D005D001F8F9CF37D03FD0089503
:10180000842F952FA62FB72FE894452B462B472BD7
:1018100011F468940895402F512F622F732F0027E1
:10182000112722273327F0E2440F551F661F771F29
:10183000001F111F221F331F081B190B2A0B3B0B04
:10184000416028F4080F191F2A1F3B1F4E7FFA958D
:1018500059F708950024E89477FF02C006D06894F1
:1018600000F809D010F80124089512D04F5F5F4F9F
:101870006F4F7F4F0895E89437FF089500951095B6
:10188000209530950F5F1F4F2F4F3F4F689408955D
:10189000409550956095709508953197F1F70895AA
:1018A000259A24982C9A239A229A8CE58CBD089527
:1018B00008950895AE2FBF2F11974A2F4B2BE1F7B4
:1018C0000895689462F80895E89462F80895EF9393
:1018D000FF93EE27E82BE92B31F0E0EAFFE03197A8
:1018E000F1F70197D1F7FF91EF910895409884E6C1
:1018F00099270E94670C409A8AE099270E94670CFA
:10190000419A81E211D080EB0FD084E00DD084E1C8
:101910000BD080E209D08CE007D00895863219F40C
:1019200081E08093D7010895429801C0429A7F9345
:1019300041988EBD90914D0097FFFCCF419A7F91C9
:10194000089500E4802FF0DF80E8EEDF882714E5BB
:10195000EDDF1A95E9F703950634A1F70895209174
:10196000D701213069F4282F203808F02FE72068AC
:1019700081E2DADF822FD8DF80E08093D7010895FB
:10198000EF93FF93509102015F9370900301E091F8
:101990000001F09101010E94750E202D0E94750E2C
:1019A000302D0E94750E002D0E94750E602D805204
:1019B000482F0E94580FE40FF51FCC241124E22E6B
:1019C000603059F1DD24DA94CD2CFF24032F0E94DE
:1019D000750E21F00A95E00FF11D03C0F3940A95EE
:1019E000B1F7FD1408F4DF2CEA9479F7E22EFF2416
:1019F000032F3197C895002021F00A95E01BF109CB
:101A000003C0F3940A95A9F7FC1408F4CF2CEA94C8
:101A100071F7D31611F4D62ECC2470920301732FD4
:101A20007C1940910301509102015F930E94670D60
:101A30005F91603041F0DD2031F05D2D0E94750E28
:101A40005A95E1F77D190E94750E802D5091040181
:101A5000513009F480954091030145350CF428D0AC
:101A6000509103015395509303017A9561F7EC0D62
:101A7000F11D603079F050910401762F88275130A4
:101A800009F4809515D0809103018395809303011B
:101A90007A95A1F7509102015395509302012A952E
:101AA00009F0BBCF5F9150930201FF91EF91089530
:101AB000213051F450910401523030F021F0509116
:101AC000030150FF01C080680E94960C08954A955A
:101AD0005A9580E229DF80E4850F26DF80E8840FB5
:101AE00023CF3C983D98449A459A08956894409332
:101AF000BC008F939F9388279927019629F04091E6
:101B0000BC0047FFFACFE8949F918F9162F8089547
:101B100044EAECDF4091B900487F483019F0403189
:101B200009F0689462F8089544E94093BC0040913C
:101B3000BC0044FDFCCF08951093BB0044E8D6DF01
:101B40008F939F9388279927019671F04091B90050
:101B5000487F483FC9F3E894483139F0483229F0CA
:101B6000403419F0403509F068949F918F9162F8E4
:101B7000089544E801C044ECB9DF1091BB004091E6
:101B8000B900487F483FD9F30895C2DF0EF40895A5
:101B90001E7FD2DF89911D91CFDF8A95E1F7C4CFF7
:101BA000122F803069F0B4DF0EF408951E7FC4DF79
:101BB000AF93BF931D91C0DF8A95E1F7BF91AF91BD
:101BC000A7DF903059F0122F1160B6DF913011F479
:101BD000D0DF01C0D0DF1D939A95C1F7A5CF8D91BD
:101BE00087FB16F48FEF01C088278D938C9308959F
:101BF0000D911D912D913C9108950191119121918B
:101C0000308108953C932E931E930E9308950F9266
:101C10001F922F92C801D901489F80014A9F9001CD
:101C20004B9F202C499F100D211D321D5A9F202CA7
:101C3000589F100D211D321D599F200D311D689F89
:101C4000200D311D699F300D789F300D2F901F9012
:101C50000F900895903041F00D911C91000F111FCD
:101C60009A95E1F71C930E930895903051F00E94DD
:101C7000F80D000F111F221F331F9A95D1F70C94F6
:101C8000020E0895903029F08C9186959A95E9F787
:101C90008C930895903041F00D911C911695079505
:101CA0009A95E1F71C930E930895903051F00E949D
:101CB000F80D36952795179507959A95D1F70C94B9
:101CC000020E0895903081F00E94F80D772737FDBD
:101CD00070E8072E000C37952795179507959A956C
:101CE000C1F7372B0C94020E0895C8953196002049
:101CF00008952E2E3F2E992781918D3209F09395CC
:101D00008823D1F79A95E22DF32D112361F009175D
:101D100018F011F0101B01C0191B28F021F080E20F
:101D20008D931A95E9F780818D3219F48D93319650
:101D300004C0222311F08BE28D93091738F031F0A3
:101D4000091B21F080E38D930A95E9F781918D932A
:101D50008823E1F7332351F0EA2FFB2F3196339597
:101D60008E9182933A95E1F78EE28C9308957F935A
:101D70000F93AF93BF938F939F938FB78F93809160
:101D8000570100E5081B29F49091C6000E94610CE0
:101D900013C000915601A5E0B1E077279091C600ED
:101DA000A00FB71F9C93839580935701039500352F
:101DB00009F40027009356018F918FBF9F918F9157
:101DC000BF91AF910F917F911895040F151F261F9A
:101DD000371F0895041B150B260B370B08950417A6
:101DE0001507260737070895000F111F221F331FFD
:101DF000089500951095209530950F5F1F4F2F4F38
:101E00003F4F0895019110810FC00E94FD0D0EC03B
:101E10000E94FD0D10C00191108117FF05C03FEF1A
:101E20002FEF04C0008111272227332737FF03C07B
:101E3000E0DF8DE28D93CF92DF92EF92AA24BB2454
:101E4000CC24DD24EE2440E2EAE0FF2755E093E3D2
:101E50008081890F87FD9F7083FD907F891B81930F
:101E60005A95A9F7C1DFAA1CBB1CCC1CDD1CEE1CBB
:101E70004A9551F7E894EFE0FF2782910CD0EB30C0
:101E8000E0F71EF068948A2D0AD088278D93EF9092
:101E9000DF90CF900895982F829501D0892F8F7071
:101EA000805D26F0803309F4089568948D93089539
:101EB000FF935527F8E0469508F4500F579547953E
:101EC000FA95D1F7FF9108952A2A2A20424D4532EA
:101ED00038302054656D70657261747572652C20A0
:101EE00048756D69646974792C20507265737375D7
:101EF00072652053656E736F72202A2A2A00232090
:101F0000424D4532383000004E6F7420666F756E5A
:101F100064210000202320424D45323830204E6F8E
:101F20007420666F756E6421000020202020202020
:101F30002020200025006800506100002054656DBD
:101F40007065726174757265203A2000204320200C
:101F5000200048756D6964697479203A2000202555
:101F6000202020005072657373757265203A20003E
:061F700020685061000032
:00000001FF
